:100000000C940F020C942C020C942C020C942C02D5
:100010000C942C020C942C020C942C020C942C02A8
:100020000C942C020C942C020C9444240C94162551
:100030000C944B1F0C942C020C942C020C942C024C
:100040000C942C020C942C020C942C020C942C0278
:100050000C942C020C94D31F0C942C020C942C02A4
:100060000C942C020C942C020C942C020C942C0258
:100070000C942C020C942C020C942C020C942C0248
:100080000C942C020C942C020C942C020C942C0238
:100090000C942C020C942C020C942C020C942C0228
:1000A0000C942C020C942C020C942C026A046A040A
:1000B00096049604FE041C05340634062705C00584
:1000C000D105D1058325AA25A226AA25A226F62593
:1000D0001926A22670267F261E001F002000A800D9
:1000E00000047F3F1F643214643214783C1E1E14D7
:1000F0000A052223252628292A2C2D2F3032333594
:1001000036383A3B3D3E4042434547494A4C4E50C3
:1001100051535557595A5C5E6062646668696B6DED
:100120006F71737577797B7D7F81838587898A8CF1
:100130008E90929496989A9C9E9FA1A3A5A7A8AAF8
:10014000ACAEAFB1B3B4B6B8B9BBBCBEBFC1C2C32D
:10015000C5C6C7C9CACBCCCDCED0D1D2D2D3D4D5C7
:10016000D6D7D7D8D9D9DADADBDBDBDCDCDCDCDCF0
:10017000DDDDDDDDDCDCDCDCDCDBDBDBDADAD9D9C8
:10018000D8D7D7D6D5D4D3D2D2D1D0CECDCCCBCA56
:10019000C9C7C6C5C3C2C1BFBEBCBBB9B8B6B4B37C
:1001A000B1AFAEACAAA8A7A5A3A19F9E9C9A989612
:1001B0009492908E8C8A89878583817F7D7B7977E5
:1001C0007573716F6D6B6968666462605E5C5A59C5
:1001D00057555351504E4C4A4947454342403E3D86
:1001E0003B3A3836353332302F2D2C2A2928262514
:1001F0002322FFAA7F5540000101010101010101F5
:1002000001020202020202020202030303030303C9
:100210000303040404040404040505050505060697
:100220000606060707070707080808080909090955
:100230000A0A0A0B0B0B0C0C0C0D0D0D0E0E0E0FFB
:100240000F0F10101111111212131314141515168B
:10025000161717181819191A1A1B1B1C1D1D1E1EFC
:100260001F2020212222232424252626272829294D
:100270002A2B2C2D2D2E2F30313232333435363778
:1002800038393A3B3C3D3E3F404142434445464776
:1002900048494A4C4D4E4F50515354555658595A4F
:1002A0005B5D5E5F616264656668696B6C6D6F70F3
:1002B00072737577787A7B7D7E8082838587888A62
:1002C0008C8E8F91939596989A9C9EA0A2A3A5A799
:1002D000A9ABADAFB1B3B5B7BABCBEC0C2C4C6C995
:1002E000CBCDCFD1D4D6D8DBDDDFE2E4E7E9EBEE4E
:1002F000F0F3F5F8FAFDFF0A03550043002D003135
:100300000000000C034D00650072006700650000EE
:10031000000403090409023B00020100A0FA0904D9
:100320000000010301010009211101000122400028
:100330000705810308000109040100010300000012
:10034000092111010001227B000705820320000121
:100350001201000200000008654D43550100010232
:10036000000105010902A10185020901A100050999
:10037000190129081500250195087501810205015B
:10038000093009311581257F9502750881060938E4
:100390001581257F950175088106050C0A3802151F
:1003A00081257F950175088106C0C005010980A1DE
:1003B00001850319012AB700150126B700950175BB
:1003C000108100C0050C0901A101850419012AA0B2
:1003D00002150126A002950175108100C0050109D2
:1003E00006A101050719E029E71500250195087503
:1003F0000181029501750881010507190029FF1582
:100400000026FF00950675088100050819012905D9
:10041000950575019102950175039101C0001124A4
:100420001FBECFEFDAE0DEBFCDBF11E0A0E0B1E04C
:10043000EAEAFFE402C005900D92A63CB107D9F7A5
:1004400022E0A6ECB1E001C01D92AC3AB207E1F7A0
:100450000E94CA110C94D3270C940000811107C08C
:10046000662311F089EA01C08AEA0E94180481E03B
:10047000089581E0089581E008950C943B02089569
:100480000C943F021F93CF93DF9300D000D01F92B4
:10049000CDB7DEB749835A836B833091C901898117
:1004A0009A81311114C0662359F0222349F00E9429
:1004B0006D08182F682F89819A810E941A0803C03D
:1004C0000E944308182F69817A81812F04C00E94FD
:1004D0006D0869817A810F900F900F900F900F90A7
:1004E000DF91CF911F910C94A20FFC01262F408128
:1004F00051816281738184810C94420281E008956C
:10050000CF93DF93EC0160E00E947502BE01DF91A2
:10051000CF910C9440020C94CC100C94C810089508
:100520000E94C4060E948F022FEF84E39CE02150BA
:1005300080409040E1F700C000000C94F91F0F9339
:100540001F93CF93DF938C0161E00E947502EC0151
:10055000B8010E943D02882309F444C0B801CE01CD
:100560000E94151E8823F1F1B801CE010E94C01B24
:100570008823C1F1B801CE010E94711D882391F139
:10058000B801CE010E94C61A882361F1F801828168
:10059000882309F1CB358DE5D807C1F050F4C1159A
:1005A000FCE5DF0781F0CF3DDC45A9F40E949E0DFC
:1005B00019C0CC35EDE5DE0761F0CD35DD4559F4E8
:1005C0000E94E70C08C00E9490020CC00E94F00C30
:1005D00002C00E94F30CC801DF91CF911F910F91CF
:1005E0000C94390280E0DF91CF911F910F91089513
:1005F0000E942C1F0E9415030C9443190E9418039B
:100600000E940F1A0C94321F08950C94040381E089
:1006100008950C9407030895CF93C82F0E940503F3
:100620008C2F0E940903CF91089580E00C940C0355
:100630000E94711E0C940C030E94711E9091C801BF
:10064000891721F08093C8010C940C030895CF936F
:10065000DF93CDB7DEB72B970FB6F894DEBF0FBE92
:10066000CDBF4F83588769877A878B8761110E9436
:10067000330C9E012F5F3F4F86E0F90111928A955E
:10068000E9F785E0FE013796D90101900D928A9530
:10069000E1F789819A814C815D81452B31F09F3F43
:1006A00031F491E08F3F19F403C091E001C090E074
:1006B00090FF09C049815A816B817C818D819E8127
:1006C0000E94540B05C0C9010E947E028111F2CF25
:1006D0002B960FB6F894DEBF0FBECDBFDF91CF9142
:1006E0000895FC01808191810E94AF080895CF9305
:1006F000882309F450C0C82F8CEF8C0F813AD0F4B6
:100700006C2F80910201909103010E94CE1E8823DC
:1007100049F06C2F80910201909103010E94061F05
:100720000E94550C6C2F80910201909103010E9450
:10073000041F0CC080E28C0F883058F4C77081E031
:1007400001C0880FCA95EAF70E94160CCF910C944D
:10075000550CEBE5EC0FE33040F4F0E0E65AFE4FC9
:10076000808190E0CF910C94961EE8E5EC0FE73184
:1007700050F4F0E0EE0FFF1FE45DFE4F80819181A9
:10078000CF910C94AC1ECD3E30F08C2F0E944F12B6
:10079000CF910C942113CF910895882389F19CEF78
:1007A000980F913A40F4682F8091020190910301D3
:1007B0000E94061F0DC090E2980F983058F4877081
:1007C00091E001C0990F8A95EAF7892F0E941C0CCD
:1007D0000C94550C9BE5980F933020F480E090E04A
:1007E0000C94961E98E5980F973120F480E090E0E5
:1007F0000C94AC1E8D3E20F00E94AA120C94211382
:1008000008951F93CF93DF93182FEB010E94770376
:10081000209741F08FE99FE00197F1F700C00000B9
:100820002197F6CF812FDF91CF911F910C94CD03AB
:10083000893319F060E070E002C060E570E00C946C
:100840000104882321F00E94160C0C94550C089585
:10085000882321F00E941C0C0C94550C0895CF9213
:10086000DF92EF92FF920F931F93CF93DF937C0160
:10087000D62FC72FFC011281058102950F700E94AF
:100880000C0C8823B9F01123A9F08C2F807F8034C1
:1008900021F080E28D0F883068F080916D0282FD3A
:1008A00009C082E00E94B50C0E940C0C91E0D82E89
:1008B000D92601C0D12CCC2EC2948FE0C8228C2D19
:1008C00090E08C30910508F0CFC1FC01EA5AFF4F4F
:1008D0000C942E278C2F807FCF70882311F0C29527
:1008E000C07F112399F0CC2309F4AAC180E28D0FB7
:1008F000883010F0D11104C08C2F0E94160C03C058
:100900008C2F0E94260C0E94550C9AC18D2F0E949C
:10091000CD03CC2309F4A8C180E28D0F883038F1D3
:10092000DD2329F18C2F0E942C0C24C08C2F807F7A
:10093000CF70803211F0C295C07FDD2319F0D13025
:10094000A1F13DC080916D0282FF17C0112349F0D3
:10095000CC2329F08C2F0E94160C0E94550C80E0AD
:1009600070C180E00E94CD03CC2309F47DC18C2F9F
:100970000E941C0C0E94550C77C1112371F00023BA
:1009800041F0013031F40E94360C8C2B0E943E0C59
:100990006BC10E94360C8C2B1DC0002319F0013056
:1009A00009F462C10E944B0C25C0112321F00630CE
:1009B00008F05AC10EC0053008F056C11BC0112303
:1009C00061F0002331F0F701858180FF39C18F701C
:1009D00085838C2F0E94210447C1002359F0D9330D
:1009E00009F03FC1FFEF07EE13E0F1500040104067
:1009F000E1F735C18C2F0E94280436C18C2F8695D3
:100A00008695837019F0813061F02EC1112321F099
:100A10008D2F9C2F937002C080E090E00E94961E64
:100A20002BC1112321F08D2F9C2F937002C080E0E9
:100A300090E00E94AC1E20C18D2F112319F00E945E
:100A40004F1202C00E94AA120E94211315C18C2FBE
:100A5000837009F047C011110BC12D2F22952695E7
:100A60002770220F220F6D2F6F70862F90E0A0E06D
:100A7000B0E0022E04C0880F991FAA1FBB1F0A9462
:100A8000D2F7D4FF10C04FE050E060E070E004C047
:100A9000440F551F661F771F2A95D2F74095509532
:100AA0006095709503C040E050E0BA01C695C695C8
:100AB000C3708A019B01082B192B2A2B3B2BC901E0
:100AC000B801C23049F058F4C13019F00E94300723
:100AD000CFC00E941E07CCC00E944207C9C00E941E
:100AE0001C07C6C0112319F08C2F817001C0869598
:100AF000882309F4BDC02D2F229526952770220F3B
:100B0000220F6D2F6F70862F90E0A0E0B0E0022ED4
:100B100004C0880F991FAA1FBB1F0A94D2F7D4FFE5
:100B200010C04FE050E060E070E004C0440F551F7B
:100B3000661F771F2A95D2F740955095609570955E
:100B400003C040E050E0BA01C695C695C3708A0163
:100B50009B01082B192B2A2B3B2BC901B801C23052
:100B600049F058F4C13019F00E94F50781C00E9485
:100B7000E3077EC00E9407087BC00E94560778C02A
:100B8000CF70112339F08C2F0E947C078D2F0E948B
:100B900021046EC08D2F0E9428048C2F0E949D0777
:100BA00067C0D23F21F128F4D03F41F0D13FC1F0DE
:100BB00043C0D33F19F1D43F79F03EC0112341F037
:100BC000053008F051C08C2F8F710E94C2074CC0B5
:100BD000063008F049C0F7CF80916D0282FF18C03F
:100BE000112339F08C2F8F710E947C073DC0112397
:100BF000C9F38C2F8F710E949D0736C0112329F0F5
:100C00008C2F8F710E9467072FC00E9462072CC033
:100C1000112349F0CF718C2F0E947C0763E08C2F49
:100C20000E949A0C21C081E00E94B50C0230E0F0D5
:100C300082E00E94B50C18C0112331F0002391F21C
:100C40008D2F0E94770310C0002399F2D93349F405
:100C50001FEF27EE33E0115020403040E1F700C095
:100C600000008D2F0E94CD0388EF8C0D843020F47E
:100C70000E94711E0E940C03DD20C9F00E94080C26
:100C800080FD15C0F70112820E94020C0E947C07B1
:100C9000C7010E9478060E94020CDF91CF911F913C
:100CA0000F91FF90EF90DF90CF900C949D07DF9114
:100CB000CF911F910F91FF90EF90DF90CF9008950B
:100CC0000F931F93CF93DF93EC01688179818A8121
:100CD0000E94BA088C010E9419080E940A07B801F4
:100CE000CE010E942F04DF91CF911F910F910895A3
:100CF000CF93DF93EC01988189812B813C81232B59
:100D000031F08F3F31F481E09F3F19F403C081E05F
:100D100001C080E080FD1DC0CE010E949F028111B4
:100D200010C00E940C0C8823A1F08A81882389F0CE
:100D300080916D0282FD0DC082E0DF91CF910C9415
:100D4000B50CCE010E946006CE01DF91CF910C94CC
:100D50008002DF91CF91089580E090E00E94961E7E
:100D600080E090E00E94AC1E0E94330C0E94550C63
:100D70000E9452140C94211380910201909103015E
:100D80000E94081F0C94AC060E94230C0C94BC0615
:100D900092959F70963079F010F4925001C09A505D
:100DA000923068F4803F69F018F4883E40F409C03E
:100DB000843F29F406C0883E20F0813F11F080E096
:100DC000089581E00895FC01808191810E94AF081F
:100DD0000E94C8060895CF93DF9300D000D01F92E1
:100DE000CDB7DEB70F900F900F900F900F90DF915F
:100DF000CF910895CF93DF9300D000D000D0CDB72E
:100E0000DEB726960FB6F894DEBF0FBECDBFDF91DA
:100E1000CF910895089508950C940B070C940C0736
:100E20000E940E076093D3017093D4018093D50183
:100E30009093D6010C94AC060C9410070F931F935B
:100E40000091D3011091D4012091D5013091D601A8
:100E5000602B712B822B932B1F910F910C941007F9
:100E60000F931F930091D3011091D4012091D501CC
:100E70003091D60160237123822393231F910F9118
:100E80000C9410070F931F930091D3011091D4017C
:100E90002091D5013091D6016027712782279327B1
:100EA0001F910F910C9410070C940B070E9454078C
:100EB0006093CF017093D0018093D1019093D201C0
:100EC0000C94AC0660E070E0CB010C9456070F93D5
:100ED0001F9341E050E060E070E08A019B0104C094
:100EE000000F111F221F331F8A95D2F7C901B801C5
:100EF0001F910F910C9456070F931F9341E050E000
:100F000060E070E004C0440F551F661F771F8A958C
:100F1000D2F78091CF019091D001A091D101B091F1
:100F2000D2018A019B01082B192B2A2B3B2BC901CB
:100F3000B8011F910F910C9456070F931F9341E036
:100F400050E060E070E004C0440F551F661F771F3B
:100F50008A95D2F740955095609570958091CF0114
:100F60009091D001A091D101B091D2018A019B0151
:100F7000082319232A233B23C901B8011F910F918C
:100F80000C9456070F931F9341E050E060E070E02F
:100F900004C0440F551F661F771F8A95D2F78091B2
:100FA000CF019091D001A091D101B091D2018A01DD
:100FB0009B01082719272A273B27C901B8011F9140
:100FC0000F910C9456070F931F930091CF0110912E
:100FD000D0012091D1013091D201602B712B822B55
:100FE000932B1F910F910C9456070F931F93009111
:100FF000CF011091D0012091D1013091D201602315
:101000007123822393231F910F910C9456070F9302
:101010001F930091CF011091D0012091D101309107
:10102000D20160277127822793271F910F910C947B
:1010300056070895990F890FE82FE695E695E695EE
:10104000877051E001C0550F8A95EAF785E0E89F67
:10105000F0011124E653FE4F20E030E070E04081C3
:10106000CB01022E02C0969587950A94E2F7817013
:10107000819584278523842781932F5F3F4F2530D7
:10108000310569F70895990F890F682F6695669560
:101090006695982F977085E0689FB001112440E015
:1010A00050E080E0FB01E40FF51FE653FE4F208186
:1010B00030E0092E02C0369527950A94E2F7217098
:1010C0003327042E01C0220F0A94EAF7822B4F5FC8
:1010D0005F4F4530510531F70895BF92CF92DF92AF
:1010E000EF92FF920F931F93CF93DF938C01C090E9
:1010F000CF01D090D001E090D101F090D201809149
:10110000D3019091D401A091D501B091D601C82A04
:10111000D92AEA2AFB2ACFE1D0E0D701C6010C2E5A
:1011200004C0B695A795979587950A94D2F780FD48
:1011300004C0219790F7B12C07C0BC2EB8018C2FAA
:101140000E94B30F0197A9F38B2DDF91CF911F91CF
:101150000F91FF90EF90DF90CF90BF900895CF93C5
:10116000DF93EC010E946D08BE010E94B30FDF9176
:10117000CF9108951F93CF93DF93EB019091C90115
:10118000992321F0CB010E94AF0813C0882349F0B6
:10119000CB010E946D08182F682FCE010E941A08FB
:1011A00004C0CB010E944308182FBE01812F0E946A
:1011B000B30FDF91CF911F9108951F93CF93DF93CA
:1011C000C091D70116E08091D801C81799F0D0E0FE
:1011D0001C9FF0011D9FF00D1124E752FE4F40812E
:1011E000518162817381848195810E94FA062196E2
:1011F000C770E9CFDF91CF911F9108954091090207
:1012000050910A0260910B0270910C0280910D02C4
:1012100090910E020C94FA06EF92FF920F931F9397
:10122000CF93DF9380910E0282958F7009F065C095
:1012300080910B02882309F460C08091D701F0905F
:10124000D8011091090200910A0260910C0270917C
:101250000D0291E01F3F09F090E0C0910001D09194
:101260000101292F96E0E92E8F1509F446C061157A
:10127000710521F00F3F21F030E003C031E001C0E3
:10128000322F90E030FD36C0E89EF001E99EF00D6F
:101290001124DF01A752BE4F11963C9111973013D4
:1012A00029C03C91311326C012963C9112973111FE
:1012B00021C013964D915C911497461B570B4C1708
:1012C0005D07C0F480910E028F70806180930E02E2
:1012D000E252FE4F80818F708061808389E092E0CE
:1012E0000E947806DF91CF911F910F91FF90EF90B0
:1012F0000C94DD0801968770B7CFDF91CF911F91D5
:101300000F91FF90EF9008959F92AF92BF92CF926E
:10131000DF92EF92FF920F931F93CF93DF93CDB79E
:10132000DEB761970FB6F894DEBF0FBECDBF8C015C
:1013300085E0F801DE011D9601900D928A95E1F796
:10134000D8011296EC9090910902E0910A02209146
:101350000C0230910D022115310531F0EF3F31F4CF
:1013600081E09F3F19F403C081E001C080E0B82F05
:10137000B1709B2E80FD47C1D8014C9111965C91B4
:1013800011971396AD90BC90149789E0C82E82E017
:10139000D82EF0900B02B501621B730B2091000157
:1013A00030910101FF2009F4D9C080910E0262172B
:1013B000730708F095C0282F207F09F052C05E13F4
:1013C00013C0491311C0FE2CE1100EC08F70806154
:1013D00080930E020E94FE08C6010E94780680914A
:1013E0000E02F80185834DC1AB2831F05F3F31F427
:1013F00081E04F3F19F403C081E001C080E080FD2F
:1014000003C081E08E2502C080E090E0F82FF170EB
:10141000FF2E80FF1CC08091D7012091D80136E0BB
:10142000821709F40BC190E0389FF001399FF00D4D
:101430001124E752FE4F6181561306C060814613A6
:1014400003C06281E61203C001968770E9CFFE2CCB
:10145000EE2009F416C180910E02816080930E0285
:1014600054C05E1306C0491304C0E11002C0F80165
:1014700099C0C8010E94E306882361F1EE2051F172
:1014800020910E02822F82958F7090E0029774F067
:101490008091090290910A0298878F831986BB86F2
:1014A000AA862C87CE0107960E94780686E0F8016E
:1014B000A9E0B2E001900D928A95E1F70E940C0933
:1014C0000E94FE080AC05E1711F1C8010E94E306DF
:1014D00081112CC0C8010E947806FF24F394D1C06A
:1014E000282F207F81F77A2DB98AA88A6E2D8989C5
:1014F0000E94EB0689E092E00E94780686E0D60121
:101500001D928A95E9F70E94FE08F12CBAC0491392
:10151000DCCFE110DACFF8018583C8010E9478069C
:1015200086E0D6011D928A95E9F7ABC0EE2091F2D4
:1015300020910E02822F82958F7090E002970CF41A
:10154000B5CF8091090290910A029A8389831B8208
:10155000BD82AC822E83CE010196A6CF621773079F
:1015600008F044C0FE2CEE2009F4B4CF5E1330C066
:1015700049132EC020910E0220FD21C0822F82959A
:101580008F70482F50E041155105C9F0F8012583AF
:101590004F30510541F08F5F982F9295907F822FA9
:1015A0008F70892B8583C8010E94780686E0F80138
:1015B000A9E0B2E001900D928A95E1F73CC086E087
:1015C000F801A9E0B2E001900D928A95E1F759C0C7
:1015D000C8010E94E306811169CF80910E028160EB
:1015E00080930E02C8010E9478064BC07A2DB98AFA
:1015F000A88A6E2D89890E94EB0686E0D6011D928D
:101600008A95E9F718C0EE2009F464CFC8010E945A
:10161000E306F82E882309F45DCF86E0F801A9E0FF
:10162000B2E001900D928A95E1F789E092E00E9484
:1016300071030E940C090E94FE0823C04D875E873B
:101640008D859E850E94AF08292F22952F7022300C
:1016500028F49F7039F0811105C00BC0243028F4A4
:101660009F7049F4805E883020F0C8010E9478069F
:101670009F2CF92C06C0D80115969C91907F91F76C
:10168000F8CF8F2D61960FB6F894DEBF0FBECDBF99
:10169000DF91CF911F910F91FF90EF90DF90CF904E
:1016A000BF90AF909F9008951F93CF93DF93CDB7D6
:1016B000DEB72C970FB6F894DEBF0FBECDBF4F83B9
:1016C000588769877A878B879C87CE0107960E9407
:1016D00084098823D1F09F8188852A853B85232B27
:1016E00031F08F3F31F481E09F3F19F403C081E076
:1016F00001C080E080FD47C04F81588569857A85AB
:101700008B859C850E94FA063EC086E0FE013796D6
:10171000DE01119601900D928A95E1F7FF81E8852F
:101720006A857B856115710531F0EF3F31F481E009
:10173000FF3F19F403C081E001C080E080FD23C0B9
:101740002091D80130E0C901019687709927409116
:10175000D70150E084179507F1F1F983EA837D837F
:101760006C8396E0929FD001939FB00D1124A752F5
:10177000BE4FFE01319601900D929A95E1F780934C
:10178000D8010E94DD0816E08091D7019091D80120
:10179000891771F1189FC001112487529E4F0E9432
:1017A0008409882329F1E091D7011E9FF0011124BB
:1017B000E752FE4F4081518162817381848195811E
:1017C0000E94FA068091D70190E0019687709927D0
:1017D0008093D701D9CF0E94C4061092D8011092ED
:1017E000D701E9E0F2E086E0DF011D928A95E9F792
:1017F0002C960FB6F894DEBF0FBECDBFDF91CF9110
:101800001F91089580911702859585958595089576
:10181000809117028770089590911702977081E068
:1018200009F480E0089580912202089590912202A7
:10183000892B80932202089580959091220289231A
:10184000809322020895109222020895909121021D
:10185000892B8093210208958095909121028923FC
:101860008093210208951092210208958091180218
:10187000089508950C94390C0C943A0C90916D02D3
:1018800092FD08C090911802981721F080931802D9
:101890000C943C0C089580911802882329F0109232
:1018A000180280E00C943C0C0895CF93DF93E091F4
:1018B0000201F0910301809122028083E0910201F4
:1018C000F0910301908180912102892B8083809186
:1018D0001802882381F0E0910201F09103019081C8
:1018E000892B808380910201909103010E94C21E86
:1018F00081110E944B0CC0910201D091030148E07C
:1019000050E06FE072E0CE010E947E27892B69F0E3
:1019100088E0FE01AFE0B2E001900D928A95E1F718
:10192000CE01DF91CF910C947D1EDF91CF91089570
:101930000C94390C90916D0292FD10C098E0899F33
:1019400090011124262B209317020E947C0780917E
:1019500017028595859585950C94980C0C947C07B9
:101960001092170280E00C94980C20911702809539
:10197000822380931702982F977099F430E0482FB4
:10198000082E000C550B2417350759F090916D0265
:1019900092FD07C08595859585950E949D070C94BD
:1019A000B00C089590916D0292FB222720F9281720
:1019B00069F080FB92F990936D0280916C02909196
:1019C0006D020E941A0D82E00C94B50C089580916E
:1019D0006D0282FB882780F991E089270C94D20C54
:1019E00081E00C94D20C80E00C94D20C80E090E06A
:1019F0000E94992721E0893E9E4F09F020E0822F26
:101A0000089582E090E00C948B2783E090E00C94A2
:101A10008B27CF9384E090E00E948B27C82F82E22F
:101A200090E00E948B272C2F30E0A901582BCA018F
:101A3000CF910895CF93C92F682F84E090E00E9442
:101A40009F276C2F82E290E0CF910C949F27AB01EF
:101A5000BC018FE090E00C94B127AB01BC0183E1A5
:101A600090E00C94B12760E070E0CB010C942D0D58
:101A700060E070E0CB010E94270D0C94330D69EEFD
:101A80007EEF80E090E00E94BD2760E082E090E081
:101A90000E949F2760E083E090E00E949F271092C1
:101AA000D3011092D4011092D5011092D60160E0BA
:101AB00084E090E00E949F2760E082E290E00E9434
:101AC0009F2760E085E090E00E949F2760E086E02D
:101AD00090E00E949F276FEF87E090E00E949F2791
:101AE00040E050E0BA0188E090E00E94B12760E059
:101AF0008DE090E00E949F2740E050E0BA0188E12D
:101B000090E00E94B12760E087E190E00E949F276B
:101B100040E050E0BA018CE190E00E94B12760E023
:101B200070E080E290E00E94BD2740E050E0BA0102
:101B300088E190E00E94B1270C94380D0C943F0D81
:101B4000682F8EE090E00C949F270E94B81F60934E
:101B50002D0270932E0280932F0290933002609397
:101B6000290270932A0280932B0290932C020895ED
:101B70000E94B81F60932D0270932E0280932F0253
:101B8000909330026093250270932602809327027F
:101B900090932802089585B7806885BF85B78068CF
:101BA00085BF089581E008950C94D20D08950C949A
:101BB000D60D0C94D60D0C94D90D0C94D60D0C9416
:101BC000DD0D0C94D60D0E94CB0D8FE890E10E94A4
:101BD000671E0E94E10D0C94DF0D0E94D70D0C943E
:101BE000D60D0E9492100C940B030E94A31F0E941A
:101BF00040110E94F10D0E94D4190E94111D0C94F5
:101C0000DB0DAF92BF92CF92DF92EF92FF920F93D4
:101C10001F93CF93DF93CDB7DEB72A970FB6F89413
:101C2000DEBF0FBECDBF0E944F11D82E81110E9482
:101C3000A50D93E2A92E92E0B92E00E010E0C02E8F
:101C4000802F0E94B610E82EF501F1905F01F82672
:101C500079F18091310281FD0E94BC10F0FC07C037
:101C6000F1FE26C0BB24B39482E0F82E03C0B12C51
:101C7000FF24F3940E94D40D882399F0BE82CF8272
:101C8000EF2081E009F480E088870E94AC1F81602A
:101C9000782F9A8789874E815F8168858A850E941F
:101CA0002703F801ED5DFD4F8081F826F08216C014
:101CB0000F5F1F4F0230110509F0C1CF8FEF8983ED
:101CC0008A831B820E94AC1F8160782F9D838C8346
:101CD00049815A816B818D810E94270381E0D11057
:101CE00001C080E02A960FB6F894DEBF0FBECDBFCC
:101CF000DF91CF911F910F91FF90EF90DF90CF90E8
:101D0000BF90AF9008950E94010E0E94181A0E9481
:101D1000241D81110E94B80D0E943F130C941C03D6
:101D2000CF93DF930E94B80FEC01811521E5920754
:101D300008F045C0811530E5930708F094C0883E4F
:101D4000910528F5803E910508F0F8C0883A910584
:101D500070F4853A910508F07CC08130910509F452
:101D600075C008F4E8C0049708F0E8C0E4C08F3BF1
:101D7000910508F0E0C0C85AD0E0CC0FDD1FC35A6F
:101D8000DE4F0990D881C02DCE019464D8C0811552
:101D900040E2940758F4811551E0950708F0CEC051
:101DA0008D3E910508F4C7C09065C9C0C11580E497
:101DB000D80708F4C0C0DF70CE01906AC0C081159A
:101DC00025E59207A8F4811534E5930708F095C03E
:101DD000811543E5940708F07BC0811552E595070E
:101DE00008F061C0D82FCC27CE01816F906AA7C0C0
:101DF000C11589E5D807A0F4C11528E5D20708F078
:101E000082C0C11536E5D30708F095C08C2F0E941B
:101E10004C108F7190E0D82FCC27CE0190628FC0EC
:101E2000C1154AE5D40708F474C0CE019056811557
:101E3000904208F080C08D2F8F710E944C10DD27DA
:101E4000D0628F71AE01582BCA0179C081E090E059
:101E500076C0C55AD0E0C557DE4F8881C82FD0E084
:101E6000CE0190646CC074E0969587957A95E1F701
:101E7000282F23703C2F337081E090E002C0880F40
:101E8000991F3A95E2F79C68AC01522B9A019C2F5E
:101E90009F709695969550E2959FE0011124C90197
:101EA0008C2B9D2B4CC08370992721E030E002C021
:101EB000220F331F8A95E2F79C2F9695969580E224
:101EC000989FE0011124C22BD32BCE019C6837C010
:101ED0008370992721E030E002C0220F331F8A95DA
:101EE000E2F79C2F9695969540E2949FE00111248D
:101EF000C22BD32BCE019A6822C0D82FCC27CE017B
:101F0000846F906A1CC0DC2FCC27CE01806F906A52
:101F100016C08C2F8F700E944C1094E0D695C795F8
:101F20009A95E1F7CF70D0E0DC2FCC27D0699E01E5
:101F3000282BC90104C080E090E001C0CE01DF91F0
:101F4000CF910895E72FF0E0E80FF11DE80FF11DA4
:101F5000EE0FFF1FE60FF11DEE0FFF1FE852FF4FC0
:101F60008591949108950E94A20F0E94900E089569
:101F70008238910569F1B0F48133910509F46DC09F
:101F800048F48932910509F463C08A32910509F455
:101F900069C008958533910509F455C089339105C9
:101FA000B9F00895833E910569F138F4803E9105BA
:101FB000B1F0823E910509F10895863E9105A9F19F
:101FC000873E9105B9F1843E910509F064C023C0B4
:101FD00020916C0220FD4FC021FD4DC008958091DD
:101FE0006C0280FD44C080916D0280FF44C08091EE
:101FF0006C0284FD42C083EE4DC080916C0282FF72
:1020000038C0F5CF80916C0282FD33C080916D02A3
:1020100080FD31C0ECCF80916D0281FF32C0809194
:102020006C0284FD2AC087EE35C080916C0283FF6C
:1020300026C0F5CF80916C0283FD21C080916D0296
:1020400081FD1FC0ECCF80916C0285FD1CC01DC0BE
:1020500080916C0285FD19C016C080916C0286FDCE
:1020600016C017C080916C0286FD13C010C089E3B2
:1020700011C082EE0FC080EE0DC080E00BC086EE76
:1020800009C084EE07C089E205C085E303C08AE287
:1020900001C081E390E0089590916C0292FF0DC021
:1020A000282F2871283019F4877F846006C0282FD4
:1020B0002471243011F48B7F886093FF0DC0282F8A
:1020C0002871283119F4877E846106C0282F247175
:1020D000243111F48B7E886120916D0220FF0DC0A8
:1020E000382F3871383019F4877F816006C0382F57
:1020F0003171313011F48E7F886021FF0DC0282F9F
:102100002871283119F4877E816106C0282F21713A
:10211000213111F48E7E886194FD877E089580E0E0
:10212000089508950E94F60C811102C00E949E0D30
:102130000E94010D809331020E94090D90936D025F
:1021400080936C020E9491100E94050D682F70E030
:1021500080E090E00E941C076091CF017091D00157
:102160008091D1019091D2010C945407E82FF0E0B6
:10217000E059FD4F80810895089580EA8A95F1F72E
:10218000089500C008950C94BD1008950C94C510D6
:102190000C94C6100C94C5100C94CA10F894E82F37
:1021A000E295EF70F0E031A1282F2F7081E090E0F0
:1021B00001C0880F2A95EAF7982F9095932391A351
:1021C00092A1892B82A37894089581E30E94CE1076
:1021D00082E30E94CE1083E30E94CE1084E30C942D
:1021E000CE10CF92DF92EF92FF920F931F93CF9377
:1021F000DF938C01C62FD0E0CE0182579E4F7C0129
:10220000FC0190819F3F99F1C62EF894E92FE29549
:10221000EF70F0E081A19F7021E030E001C0220F5B
:102220009A95EAF7822B81A382A12095282322A3E5
:1022300078940E94C110D3B01C9902C082E001C002
:1022400080E0D3FADD24D0F891E0D926D82AF7012E
:1022500080818F3F11F00E94CE1061E0D11001C04B
:1022600060E08C2D0E94C310C00FD11FD882DF9177
:10227000CF911F910F91FF90EF90DF90CF90089535
:102280000E94E510109271021092700210926F027B
:1022900010926E0282E00E9487110C948B021F93B1
:1022A000CF93DF9300D0CDB7DEB71A82198260E0FA
:1022B000CE0101960E94F11061E0CE0101960E94CC
:1022C000F11042E050E0BE016F5F7F4F8EE692E07A
:1022D0000E947E2711E0009709F410E0892B31F06D
:1022E00089819A8190936F0280936E02212F42E040
:1022F00060E772E08EE692E00E9488110E948D02F3
:10230000812F0F900F90DF91CF911F910895089525
:10231000FF920F931F93CF93DF938C01F62ED72F4D
:10232000C42F222349F081E0809334020E94AC1F25
:102330009093330280933202809134028823C1F05B
:1023400080913202909133020E94C41F059780F061
:10235000EF2DFD2FD8014C2F50E0CD01801B910BAC
:10236000841795071CF48D918193F7CF1092340256
:10237000DF91CF911F910F91FF9008950E949C21B2
:102380000E94F50D0C94A8210E94AC210E94830E9E
:102390000C94C6210E944A1F0E9483210E94E30DD3
:1023A0000E94BE110E94C4110E94ED0DFBCF8091CE
:1023B0003B0280FF06C06091090170E0660F771F45
:1023C00026C081FF04C06091090184E005C082FF3E
:1023D00007C06091090188E0689FB001112417C00F
:1023E00090913A029923D1F060910801961788F7ED
:1023F0002091090188E0289F90011124929FA0015B
:10240000939F500D112470E0CA010E94F826603895
:10241000710540F46115710519F406C068E070E0BB
:10242000862F08958FE7089581E0089580913B02FB
:1024300080FF08C06091050170E0759567957595FE
:10244000679521C081FF06C06091050170E0759518
:10245000679519C082FF04C06091050170E010C04B
:1024600090913902992399F0609104019617A0F791
:1024700080910501899FC001112470E00E94F82617
:102480006038710540F46115710519F406C061E00A
:1024900070E0862F08958FE7089581E008958D3EBE
:1024A00021F40E94D711819504C08E3E29F40E9428
:1024B000D71180933F0208958F3E21F40E94D711D7
:1024C000819504C0803F29F40E94D71180933E0279
:1024D0000895893F19F40E94161205C08A3F31F40D
:1024E0000E94161281958093400208958B3F21F43B
:1024F0000E941612819504C08C3F29F40E94161286
:102500008093410208959FE0980F983078F421E07D
:1025100030E0A90102C0440F551F9A95E2F7CA01A5
:1025200090913D02892B80933D0208958D3F21F4C7
:1025300080913B0281600BC08E3F21F480913B0271
:10254000826005C08F3F29F480913B0284608093B4
:102550003B0208958D3E39F490913F0297FF35C0BC
:1025600010923F0259C08E3E29F490913F021916F5
:10257000BCF32BC090913E028F3E29F497FF25C0FB
:1025800010923E0249C0803F19F41916CCF31DC0C9
:1025900090914002893F29F41916BCF41092400230
:1025A0003BC08A3F19F497FF10C0F8CF8B3F39F436
:1025B0009091410297FF09C0109241022DC08C3FBB
:1025C00021F4909141021916BCF39FE0980F9830C6
:1025D00080F421E030E0A90102C0440F551F9A9514
:1025E000E2F7CA01809590913D02892380933D02D4
:1025F00013C08D3F21F480913B028E7F0BC08E3F34
:1026000021F480913B028D7F05C08F3F29F480919A
:102610003B028B7F80933B0280913E02811106C07A
:1026200080913F02811102C010923A0280914002D3
:10263000811106C080914102811102C010923902BD
:1026400008950E94AC1F20913E02211104C02091E8
:102650003F02222321F09093380280933702209189
:102660004002211104C020914102222321F09093C5
:102670003602809335028CE392E00C94881EEF9230
:10268000FF920F931F93CF93DF9300D000D000D021
:10269000CDB7DEB786E0ECE3F2E0DE011196019003
:1026A0000D928A95E1F7E0903E02F0903F02009192
:1026B00040021091410210923E0210923F0210928D
:1026C000400210924102E11003C0FF2009F45DC0F6
:1026D00080913702909138020E94C41FAC01909102
:1026E0003A02992339F020910A0130E02417350786
:1026F00058F04BC020910B018AE0289F90011124D3
:102700002417350718F041C09F3F19F09F5F909341
:102710003A02EE2061F00E94D7111E1414F09FEFD0
:1027200001C091E0989F902D112490933E02FF20CC
:1027300061F00E94D7111F1414F09FEF01C091E0C7
:10274000989F902D112490933F0230913E023323A5
:10275000E1F020913F022223C1F045EB3403C00198
:102760001124992319F090933E0203C081E08093D5
:102770003E0235EB2303C0011124992319F09093F5
:102780003F0203C081E080933F02011103C0112387
:1027900009F45DC080913502909136020E94C41FF9
:1027A000AC0190913902992339F02091060130E073
:1027B0002417350758F04BC0209107018AE0289F65
:1027C000900111242417350718F041C09F3F19F0DC
:1027D0009F5F90933902002361F00E941612101639
:1027E00014F09FEF01C091E0989F902D11249093D9
:1027F0004002112361F00E941612111614F09FEF8F
:1028000001C091E0989F902D112490934102309146
:1028100040023323E1F0209141022223C1F045EB35
:102820003403C0011124992319F09093400203C08E
:1028300081E08093400235EB2303C00111249923EA
:1028400019F09093410203C081E08093410280918E
:102850003E0281110BC080913F02811107C080911F
:102860004002811103C08091410281110E94211315
:10287000EB82FC820D831E8386E0FE013196ACE381
:10288000B2E001900D928A95E1F726960FB6F89482
:10289000DEBF0FBECDBFDF91CF911F910F91FF9093
:1028A000EF900895ECE3F2E086E0DF011D928A9557
:1028B000E9F710923A021092390210923B02089501
:1028C000EF92FF920F931F93CF93DF938B01682FAB
:1028D00011110AC0442329F0E82FF0E0E950FE4F1F
:1028E0006491762F862F75C0212F30E0E82FF0E01D
:1028F000442321F0E950FE4FE491F0E046E0049FCC
:10290000C0011124CFEFD0E0BE010E94E4264BEAC3
:102910004603C001479F900D1124800F911D800F29
:10292000911D982F990F890FAE01421B530B4E9F9B
:10293000D0014F9FB00D5E9FB00D11249B2F189FAB
:10294000A0011124452F55278E01041B150B0E9F46
:10295000A0010F9F500D1E9F500D11247E01E81AFB
:10296000F108E29E8001E39E100DF29E100D1124ED
:10297000212F3327C21BD30BCE9F9001CF9F300D49
:10298000DE9F300D112462307105A9F048F4611505
:10299000710569F061307105C9F48B2F752F0DC079
:1029A0006430710581F058F06630710579F47E2F3E
:1029B0008B2F932F0DC0832F7B2F9E2F09C08E2F1F
:1029C0007B2F952F05C08E2F732F02C07E2F852F52
:1029D000692FDF91CF911F910F91FF90EF90089594
:1029E00041E00E946014089508950E94F014089533
:1029F000CF93DF93762FE901682F842F0E94F5147F
:102A0000798368838A83DF91CF91089580917202E0
:102A1000282F269530E02115310519F48170826048
:102A200005C02532310524F08170886480937202DC
:102A3000089588E090E00C949327CF92DF92EF9274
:102A4000FF926B017C010E940615B701A60188E088
:102A500090E0FF90EF90DF90CF900C94B127E2E7E9
:102A6000F2E083E0808311828FEF8283838314827C
:102A700060817181828193810C941D158091720215
:102A800080FF02C08695089580E0089590917602B7
:102A9000933018F49F5F90937602882351F06091F1
:102AA00072027091730280917402909175020C947D
:102AB0001D15089581E00C94461590917602992396
:102AC00019F0915090937602882351F06091720230
:102AD0007091730280917402909175020C941D158F
:102AE000089581E00C945D1570E00C94951B609145
:102AF00010018091720280FF0AC080910F0123E0D3
:102B0000829FC001112489589D4F0C9474158091A7
:102B1000110190911201891780F7E82FF0E09F01D1
:102B2000220F331FE20FF31FE958FD4F118210826D
:102B300012828F5FF0CF9091720290FF16C0909139
:102B4000110120911201921770F4E92FF0E0DF01DA
:102B5000AA0FBB1FEA0FFB1FE958FD4F818360835B
:102B600042839F5FF0CF0C9477150895CF93DF9346
:102B700000D01F92CDB7DEB79091720290FF0AC0CD
:102B80009E012F5F3F4F0E94F8144B8169818A811B
:102B90000E949B150F900F900F90DF91CF91089599
:102BA000CF93DF93EC01EC81F0E0EE50FF4F4491C6
:102BB000E2E7F2E0628181810E94B6158C818F5F2D
:102BC0008C83DF91CF910895CF93DF93EC01E2E7FF
:102BD000F2E0438162818C810E94B6158C818F5F07
:102BE0008C83DF91CF9108950F931F93CF93DF9341
:102BF00000D01F92CDB7DEB78C01809142028111C7
:102C00000AC09E012F5F3F4F4FEF6FEF0E94F814F5
:102C10008A8180934202F8018481813051F028F04A
:102C2000823061F4409142020AC08091420240E049
:102C300007C06091420240E080E003C040E080E0D5
:102C400060E00E949B15F801848190E0019663E0AA
:102C500070E00E94F82684830F900F900F90DF9110
:102C6000CF911F910F910895AF92BF92CF92DF92B3
:102C7000EF92FF920F931F93CF93DF9300D01F9299
:102C8000CDB7DEB7182FF62E042FE22E90917202E8
:102C900090FF6DC0E92FE695AE2FB0E0A057BE4F74
:102CA0008C9180934E029E7F923061F49E012F5F43
:102CB0003F4F812F0E94F8144B8169818A810E94C5
:102CC0009B1543C0823019F4009175023EC08630D6
:102CD00019F41091730239C08930D9F38931A9F5FB
:102CE000E9518E2F8170D82EE695F0E0EE50FE4F20
:102CF000A590B490C12CBB2460911301C61618F5A1
:102D00002C2D30E0A29EC001A39E900DB29E900D8E
:102D1000112470E00E94E426812FD11002C0860F9A
:102D200001C0861B90911101290F311DA901440F8B
:102D3000551F240F351F29583D4F402F6F2D0E94DE
:102D4000F814C394D9CF0E94771510937302F092B0
:102D5000740200937502EE2051F06091720270913E
:102D6000730280917402909175020E941D150F905C
:102D70000F900F90DF91CF911F910F91FF90EF90E7
:102D8000DF90CF90BF90AF900895E2E7F2E091819D
:102D9000282F438162818AE0890F0C94341681E0E8
:102DA0000C94C516E2E7F2E09181282F43816281FD
:102DB00086EF890F0C94341681E00C94D216E2E76A
:102DC000F2E062812AE0620F08F46FEF282F43815E
:102DD00081810C94341681E00C94DF16E2E7F2E076
:102DE00062812AE0621B08F460E0282F4381818120
:102DF0000C94341681E00C94EE16E2E7F2E0438185
:102E00002AE0420F08F44FEF282F628181810C9451
:102E1000341681E00C94FD16E2E7F2E043812AE0EB
:102E2000421B08F440E0282F628181810C94341603
:102E300081E00C940C1720E00C943416FF920F9351
:102E40001F93CF93DF93EC01F12C0FEF10E0609113
:102E50001301F616F0F4809111012F2D30E0280FA8
:102E6000311DC901880F991F280F391F29583D4F5F
:102E700070E0C8010E94F826962F8C81409175025F
:102E800060917402F99E800D11240E94F814F3944D
:102E9000DECF0E9477159A818C8190FF02C08F5FF0
:102EA00001C081508C83DF91CF911F910F91FF90D2
:102EB0000895AF92BF92CF92DF92EF92FF920F935D
:102EC0001F93CF93DF93FC01828180FF02C00FEF3D
:102ED00001C001E010E04CE0A42E8091130118170E
:102EE00008F043C080911101C12ED12CE601C80F1A
:102EF000D11DCE01880F991FC80FD91FC958DD4FAA
:102F0000198218821A8234E0E32EF12CB12C8091C0
:102F100044028B0D8D302CF06A2D0E94D626892F0D
:102F200005C087FF03C090911301890F082E000C84
:102F3000990BC816D90691F4809175028E9DA00157
:102F40008F9D500D112455954795559547959E0198
:102F500060917402809173020E94F814B00EF1E047
:102F6000EF1AF108A1F61F5FB8CF0E947715809184
:102F70004402013031F4811102C08091130181506B
:102F800007C090E001966091130170E00E94F8265E
:102F900080934402DF91CF911F910F91FF90EF90AA
:102FA000DF90CF90BF90AF900895CF9380911101A3
:102FB00090911201891770F4E82FF0E09F01220F21
:102FC000331FE20FF31FE958FD4F11821082128266
:102FD0008F5FF0CFC0E060911301C617C0F5EC2FF2
:102FE000F0E070E0CF010E94F82620911101820FDD
:102FF00020914302022E000C330B90E0E217F307FE
:10300000CCF020910E01022E000C330B2E173F073F
:103010008CF09C01220F331F820F931F9C012958B3
:103020003D4F4091750260917402809173020E943D
:10303000F8140BC0FC01EE0FFF1F8E0F9F1FFC0149
:10304000E958FD4F118210821282CF5FC4CF0E94D7
:10305000771520910D0180914302820F80934302E6
:1030600090910E01920F90930E0119165CF4082EA8
:10307000000C990B4091130150E041505109841705
:1030800095071CF0219520930D01CF9108958F9203
:103090009F92AF92BF92CF92DF92EF92FF920F93E7
:1030A0001F93CF93DF938C01FC014481C42FD0E0A8
:1030B0009E01DE010E943C279B01AC010E94522729
:1030C0006B017C01E0E2F0E0EC1BFD0BA5E5B0E05C
:1030D0009B01AC010E9452274B015C019F01DF0163
:1030E0000E9434279B01AC010E945D279B01AC012B
:1030F0002C0D3D1D4E1D5F1DC501B4010E940C2706
:10310000C22FD22F2A3228F4F3E02F9F90011124EE
:103110000DC025E530E02C1B3109C901880F991F2E
:10312000280F391F37FF02C02F5F3F4F3595279576
:10313000C22FC095F12C85E5E82EED1A8091130180
:10314000F816C8F4F1FC02C08E2D01C08D2F9091AD
:1031500011012F2D30E0290F311DA901440F551FFA
:10316000240F351F29583D4F4C2F609174020E9447
:10317000F814F394E3CF0E947715F801848181114C
:1031800002C091E003C0803219F49FEF90930C01CC
:1031900090910C01890FF8018483DF91CF911F91E9
:1031A0000F91FF90EF90DF90CF90BF90AF909F90E6
:1031B0008F9008950F931F93CF93DF93EC0100E05E
:1031C00010E080911301282F30E00217130724F537
:1031D000909111019801290F311DA901440F551F2C
:1031E000240F351F29583D4F869590E04C810817D4
:1031F00019071CF4442331F002C0411103C040916F
:10320000750201C040E060917402809173020E94D7
:10321000F8140F5F1F4FD5CF0E9477158C8190E077
:103220000196817099278C83DF91CF911F910F9127
:103230000895E2E7F2E080818E7F80836081718172
:10324000828193810E941D1510924F022FEF80E71B
:1032500092E0215080409040E1F700C000000C94C3
:103260007715E2E7F2E080818E7F808310924F0233
:103270002FEF80E792E0215080409040E1F700C0BE
:1032800000000C94771510924F0280914C0281112E
:103290000AC081E080934C02809172028170809319
:1032A0004B020C943119089560917202669570E09A
:1032B0004BE050E084E191E00E947127892B19F4E2
:1032C00081E080934F020E94AC1F9093460280934E
:1032D000450208959091720290FF35C0917081115E
:1032E00002C0926006C0853210F0986402C0880F58
:1032F000982B90937202662351F060917202709144
:10330000730280917402909175020E941D15609164
:103310007202669570E04BE050E084E191E00E941B
:103320007127892B19F010924F0202C00E94541984
:1033300081E080934802409175026091740280910F
:1033400073020C941B170895682F90917202969542
:1033500081E0890F853208F081E00C946A1981E0E0
:103360000C94A419682F9091720296958FEF890F93
:1033700009F484E20C946A1981E00C94B21961E0BA
:103380000C946A19E2E7F2E080818160808386957F
:103390000C94BF198091720280FD0C9419190C9441
:1033A000C21960E00C946A1980914D0281112EC0FF
:1033B0000E94F60C811104C00E949E0D0E942F15E0
:1033C0000E941915609372027093730280937402C5
:1033D000909375026E7F61F40E942F150E9419155B
:1033E00060937202709373028093740290937502DB
:1033F0000E94061510924F028091720280FF03C056
:1034000086950E94D11981E080934D020895E2E7EC
:10341000F2E080818160808386950C94D1191092AE
:103420004C0280914B0281110E94071A0C9454198E
:103430000F931F93CF93DF9380914F02882309F45A
:1034400085C080914E02E0917202E695E81BE09300
:103450004702823049F4F0E0E251FF4FE491CE2F71
:10346000D0E000ED15E149C0863049F4F0E0E551C7
:10347000FF4FE491CE2FD0E004EE15E13EC089303D
:1034800051F4E695F0E0E851FF4FE491CE2FD0E003
:103490000EE117E132C08F3051F4E695F0E0EB51C8
:1034A000FF4FE491CE2FD0E009E517E126C085312A
:1034B00049F4F0E0EE51FF4FE491CE2FD0E005ED5E
:1034C00017E11BC0883181F0833239F4E0EEF0E07F
:1034D000C591D49104EF15E110C0843251F4C4EFCA
:1034E000D1E00AED18E109C0C8E2D0E007E418E134
:1034F00004C0C0EDD7E004EF14E1809148028823B6
:1035000061F0109248020E94AC1F90934602809393
:10351000450210924A02109249020E94AC1FE091AB
:103520004502F09146028E1B9F0B8F3F9F4770F420
:10353000EC0FFD1FF0934602E093450285E492E014
:10354000F801DF91CF911F910F910994DF91CF91F5
:103550001F910F910895882311F0FA0101C0FB011A
:103560000994CF93DF93C82FD62F0E943E158C1756
:1035700040F00E943E158D1720F4DF91CF910C94FE
:10358000AF198C2FDF91CF910C94BF191F93CF935C
:10359000DF93FB0112811111C3C0EC010E94130CD7
:1035A0008272CD3CFCE5DF0709F49AC0A8F5C73C60
:1035B000ECE5DE0709F476C0A8F4C43C9CE5D90725
:1035C00009F45FC028F4C33CDC4509F457C054C07B
:1035D000C53C9CE5D90709F459C0C63CDC4509F453
:1035E0005CC04AC0CA3CFCE5DF0709F46AC050F47D
:1035F000C83CECE5DE0709F45AC0C93CDC4509F4D7
:103600005BC03AC0CB3C9CE5D90709F45FC0CC3C19
:10361000DC4509F460C030C0C23DFCE5DF0709F4B9
:103620006FC088F4CF3C9CE5D90709F460C008F46A
:103630005CC0C03DFCE5DF0709F45CC0C13DDC4572
:1036400009F45BC019C0C53D9CE5D90709F460C009
:1036500050F4C33DFCE5DF0709F455C0C43DDC452B
:1036600009F454C009C0C63D9CE5D90709F455C00A
:10367000CE35DD4509F454C011E052C00E94CA198C
:103680004FC04CEB59E16FEA79E104C04FEA59E1D0
:103690006CEB79E10E94AB1A43C04CED56E16FEC44
:1036A00076E1F8CF4FEC56E16CED76E1F3CF4AEFDF
:1036B00056E16BEE76E1EECF4BEE56E16AEF76E146
:1036C000E9CF48E157E169E077E1E4CF49E057E12C
:1036D00068E177E1DFCF41E755E16AE575E1DACFEF
:1036E0004AE555E161E775E1D5CF81E017C065E0B6
:1036F00082E010C068E086E00DC06EE089E00AC09C
:1037000064E18FE007C067E185E104C088E106C09D
:1037100062E289E10E94B11A03C083E20E94BF19EC
:10372000812FDF91CF911F910895259A25B12F7D8B
:1037300035B130624FB7F894FC01CB01880F991F67
:10374000680F791F6E0F7F1FE617F70789F08191C9
:1037500098E035B9000000C087FF25B9880F000048
:1037600000C000C000C025B900C09A9591F7ECCF09
:103770004FBF8FE594E00197F1F700C00000089576
:10378000CF93DF93EC01FB018281882309F43CC1D4
:10379000C430FDE5DF0760F4CB3F9CE5D90788F432
:1037A0009E0122503C452431310508F02EC109C04C
:1037B000C236EDE5DE0729F0C63AFDE5DF0709F080
:1037C00024C10E94090D90936D0280936C02C13157
:1037D0008CE5D80709F4C6C008F042C0C930ECE552
:1037E000DE0709F49BC000F5C5308CE5D80709F465
:1037F00085C078F4C330ECE5DE0709F478C008F042
:103800007AC0C230DC4509F0F5C080916C0281605D
:10381000EFC0C7309CE5D90709F478C008F07AC03A
:1038200080916C028061E4C0CD30FCE5DF0709F4D3
:1038300087C058F4CB309CE5D90709F479C008F06B
:103840007BC080916C0288606FC0CF30FCE5DF07E1
:1038500009F480C008F082C080916C02877FC8C0E4
:10386000CE3F9CE5D90709F471C000F5C531FCE5F0
:10387000DF0709F485C068F4C3319CE5D90709F472
:1038800075C008F095C00E94C40680916C028F77C5
:10389000AFC0CC3FFCE5DF07A9F108F054C0CB3F37
:1038A000DC4509F0A7C080916D0240C0C230EDE553
:1038B000DE0709F489C058F4C1158DE5D80709F46D
:1038C0005AC008F069C080916D0282602FC0C23674
:1038D000EDE5DE0709F47CC0C63AFDE5DF0709F433
:1038E00081C0C330DD4509F085C080E06EC08091A5
:1038F0006C0282607DC080916C0216C080916C0267
:10390000886076C080916D0282604FC080916C02A9
:1039100080626EC080916C0280646AC00E94C4069E
:1039200080916C02806864C0846062C081603DC028
:1039300080916C028E7F5CC080916C028D7F58C03C
:1039400080916C0216C080916D0218C080916D024A
:103950008D7F2BC080916C028F7E4AC080916C025B
:103960008F7D46C080916C028F7B42C080916C023B
:10397000877F8B7F3DC080916D028D7F8E7F15C0CC
:1039800080916C0282FB222720F991E0922790FB24
:1039900082F990FB83F92CC080916D02982F90954D
:1039A00091708E7F892B90FB81F980936D0222C0EC
:1039B0000E94C40680916C0287FB222720F991E0C7
:1039C000922790FB87F914C081E00E94A00D12C0DD
:1039D00080916C0284FB222720F991E0922790FBD2
:1039E00084F906C080916C02982F909590FB80F925
:1039F00080936C0280916C0290916D020E941A0D6E
:103A00000E94C40680E001C081E0DF91CF9108955B
:103A10008FE891E00197F1F700C0000008950C9441
:103A20002E0285988D9A86988E9A0E94081D8FB1D5
:103A300085FB882780F97E9902C090E001C092E062
:103A4000892B809352020895E0915202EE0FEE0FFF
:103A5000E09352024FB145FB882780F990E04FB1C7
:103A600046FB222720F930E046FF02C022E030E08A
:103A7000822B932B8E2B809352028F70E82FF0E0D5
:103A8000EB54FE4F908180915102890F8093510237
:103A900084305CF0809150028F5F8093500260E030
:103AA00080E00E940F1D21E001C020E080915102C2
:103AB0008D3F54F48091500281508093500261E018
:103AC00080E00E940F1D21E080915102082E000C21
:103AD000990B64E070E00E94F82680935102822FD7
:103AE0000895CF93DF9386319C4541F5EB010E9409
:103AF000130C982F8A8120910201309103018823B1
:103B000079F09A7A81E009F480E080935302911170
:103B100002C069E201C065E3C9010E94041F0AC036
:103B200080915302811102C069E201C065E3C901BD
:103B30000E94061F0E94550C80E001C081E0DF91C9
:103B4000CF9108950F931F93CF93DF93C42FD22F5C
:103B5000FC0182818823C9F0409356020E94AC1F69
:103B6000909355028093540280E28C0F883008F0C5
:103B700057C0C77081E001C0880FCA95EAF7DF918E
:103B8000CF911F910F910C942104809156024813FC
:103B900030C080915402909155020E94C41F883C0D
:103BA000910538F510E21D0FCD17B9F080E28C0FAA
:103BB000883040F4C77081E001C0880FCA95EAF7E9
:103BC0000E942804183028F581E09D2F977001C0CD
:103BD000880F9A95EAF70E942104802F0E9418040A
:103BE0001830F0F4D77081E001C0880FDA95EAF759
:103BF0000AC080E28C0F883098F4C77081E001C061
:103C0000880FCA95EAF7DF91CF911F910F910C941D
:103C10002804802FDF91CF911F910F910C941804ED
:103C2000DF91CF911F910F9108950F939C01CB01CC
:103C3000243F4CE5340731F188F4293DFCE53F078A
:103C4000D9F02A3D4CE5340779F1283D3C45A9F5EA
:103C500006E221EE41EE68ED7CE52BC0263FFCE557
:103C60003F07E1F0A8F0273F3C4539F507E225EE94
:103C700046EE67EF7CE51DC007E225EE45EE69EDF7
:103C80007CE517C006E221EE40EE64EF7CE511C052
:103C900007E225EE44EE65EF7CE50BC006E221EE7F
:103CA00042EE66EF7CE505C008E221E045EE6AEDF4
:103CB0007CE50E94A21D80E008C0FC01828188236F
:103CC00019F01092560201C081E00F91089590936F
:103CD000C7018093C601089590935C0280935B02B4
:103CE0000895E0915B02F0915C02309721F0019021
:103CF000F081E02D099480E00895E0915B02F0915D
:103D00005C02309721F00280F381E02D0994089540
:103D1000E0915B02F0915C02309739F022E0DC0127
:103D20002C930480F581E02D099408952091590287
:103D300030915A022817390771F090935A028093F4
:103D40005902E0915B02F0915C02309721F006800D
:103D5000F781E02D0994089520915702309158027F
:103D60002817390771F09093580280935702E09119
:103D70005B02F0915C02309721F00084F185E02D28
:103D800009940895FC01329697E080E0915029F063
:103D900021912223D9F38F5FF9CF0895662349F04B
:103DA000FC01329608962191621729F0E817F9076D
:103DB000D1F780E0089581E008959C01FC013296DE
:103DC0009FEF80E04191461789F09F3F19F4411120
:103DD00001C0982F8F5F8630A9F79F3F39F0F90116
:103DE000E90FF11D97FDFA956283089508959C01EE
:103DF0002A5F3F4FFC014281461301C012820196A7
:103E000082179307B9F708950C94DD1E0C94F71EE2
:103E1000029626E0FC0111922A95E9F7089508958B
:103E20000C940F1F83E080935D020C94101F81118E
:103E300002C081E001C082E080935D020C94101FFB
:103E40000C94171F81E080935D020C94101F0C945A
:103E5000221F08950C94291F0C942A1F0C94291FCB
:103E60000C94291F0C94291F0E94301F0E944F118F
:103E70000E942E1F80E00E94B610811108C081E0D0
:103E80000E94B61091E0811103C090E001C091E062
:103E9000892F089508951F920F920FB60F92112443
:103EA0008F939F93AF93BF9380915E02811113C054
:103EB00080919B0290919C02A0919D02B0919E02E4
:103EC0004196A11DB11D80939B0290939C02A093EB
:103ED0009D02B0939E02BF91AF919F918F910F90E1
:103EE0000FBE0F901F9018958091A302843031F17E
:103EF0000E94F80210925E0220E488E190E00FB682
:103F0000F894A895809360000FBE2093600083B75B
:103F1000817F846083BF83B7816083BF78948895F5
:103F200083B78E7F83BF0FB6F894A8958091600009
:103F3000886180936000109260000FBE08950E9417
:103F4000C4060C94FE0282E084BD93E095BD9AEF16
:103F500097BD80936E0008952FB7F89480919B02CF
:103F600090919C02A0919D02B0919E022FBF089556
:103F70002FB7F89460919B0270919C0280919D02F2
:103F800090919E022FBF08959C014FB7F8948091A5
:103F90009B0290919C02A0919D02B0919E024FBF06
:103FA000821B930B089578941F920F920FB60F9275
:103FB00011248F939F93AF93BF9380919B02909115
:103FC0009C02A0919D02B0919E020196A11DB11D7F
:103FD00080939B0290939C02A0939D02B0939E02BB
:103FE000BF91AF919F918F910F900FBE0F901F9037
:103FF000189587E797E790930108809300089AE067
:1040000088E10FB6F894A895809360000FBE909356
:104010006000FFCF80916A020895089522E0209306
:10402000E9002FEF3091E800215035FD06C035ED55
:104030003A95F1F700002111F5CF2091E80025FF16
:104040000BC040E050E066E070E00E9438228091B2
:10405000E8008E778093E8000895CF93DF9321E006
:104060002093E9002FEF3091E800215035FD06C084
:1040700035ED3A95F1F700002111F5CF2091E800D8
:1040800025FF14C0EC0140E050E068E070E00E94C1
:1040900038228091E8008E778093E80088E0FE0166
:1040A000A2E6B2E001900D928A95E1F7DF91CF91FF
:1040B000089580935F027093610260936002809123
:1040C000A302843001F582E08093E9008FEF9091A4
:1040D000E800815095FD06C095ED9A95F1F7000036
:1040E0008111F5CF8091E80085FF0DC040E050E0E0
:1040F00063E070E08FE592E00E9438228091E80052
:104100008E778093E8000895BC0184E00C945920D8
:10411000BC0183E00C9459208091A202811109C056
:104120000E94C9230E9426248091E200846080932B
:10413000E20008951092A20208950C94271F609146
:104140009F0281E0611101C080E00C94121F9091E8
:10415000A30281E0943009F080E060919F020C940A
:10416000171F42E061EC81E00E94422342E261ECD1
:1041700082E00E9442239091A30281E0943009F0F2
:1041800080E060919F020C94201F8091A5028330F3
:1041900009F461C030F4813071F0823009F49AC0C2
:1041A00008958A3009F486C08B3009F46CC08930D8
:1041B00009F0A8C020C08091A402813A09F0A2C0F1
:1041C0008091E800877F8093E8008091A802909119
:1041D000A902892B21F468E082E692E003C060E046
:1041E00080E090E070E00E9483228091E8008B776D
:1041F0008093E80008958091A402813209F082C082
:104200008091A8029091A902029708F07BC080914A
:10421000E800877F8093E8008091E80082FD05C078
:104220008091A3028111F8CF6DC02091F30080919D
:10423000F20090E0922B029731F48091F1008130EE
:1042400011F0863021F48091F10080936A02809110
:10425000E8008B7753C08091A402813A09F052C0E4
:104260008091A8029091A902892B09F04BC08091FE
:10427000E800877F8093E8008091E80080FFFCCF12
:1042800080912B0136C08091A4028132D9F58091B2
:10429000A8029091A902892BA9F58091E800877F57
:1042A0008093E8000E9477238091A60280932B01DF
:1042B0000C94C4068091A402813221F58091E8001B
:1042C000877F8093E8000E9477238091A7028093E4
:1042D0006B0208958091A402813AA1F48091E800D4
:1042E000877F8093E8008091E80080FFFCCF809179
:1042F0006B028093F1008091E8008E778093E80054
:104300000C947723089584B7877F84BF0FB6F89401
:10431000A895809160008861809360001092600091
:104320000FBE90E080E80FB6F89480936100909300
:1043300061000FBE0C94221F0E94C9230E942624F4
:10434000E2EEF0E080818460808378940C94BB2658
:104350008FE191E00C946C1E8091A3028530A9F44A
:104360008091A302853079F40E94741F8091A1028C
:104370008823B1F30E94341F882391F30E942222E4
:104380000E94C406EDCF0C949F1F089508950C94CD
:10439000C921292F332723303105C9F060F421309A
:1043A000310581F02230310509F044C08BE390E003
:1043B00025E133E043C021323105E1F022323105FD
:1043C00049F138C082E190E020E533E037C0992719
:1043D0008130910549F028F0029761F5E7EFF2E0AE
:1043E00005C0E1E1F3E002C0E3E0F3E0849190E096
:1043F0009F0124C06115710541F061307105D1F450
:1044000089E090E020E433E019C089E090E027E201
:1044100033E014C06115710541F06130710551F44C
:104420008BE790E022E633E009C080E490E02DEDD8
:1044300033E004C080E090E020E030E0FA01318316
:104440002083089580E189BD82E189BD09B400FE21
:10445000FDCF8091D8008F7D8093D8008091E000BF
:1044600082608093E0008091E00081FDFCCF0895A0
:10447000CF92DF92EF92FF920F931F93CF93DF9330
:10448000EC018B017A010E949623811133C0E11463
:10449000F10439F0F70180819181081B190BC80FD5
:1044A000D91FC12CD12C0115110519F18091E800FB
:1044B00085FD16C08091E8008E778093E800E114B6
:1044C000F10449F0F70180819181C80ED91ED18293
:1044D000C08285E00FC00E949623882321F30AC082
:1044E00089918093F10001501109FFEFCF1ADF0A83
:1044F000DACF80E0DF91CF911F910F91FF90EF9085
:10450000DF90CF9008952091AA023091AB02261738
:10451000370748F06115710539F42091E8002E77CE
:104520002093E80001C0B901FC0120E0611571058C
:1045300079F18091A3028823F1F18530F1F1809126
:10454000E80083FD3CC08091E80082FD2EC0809190
:10455000E80080FFEBCF2091F3008091F20090E023
:10456000922B6115710551F08830910538F4219135
:104570002093F100615071090196F3CF21E0089773
:1045800009F020E08091E8008E778093E800CECF9C
:104590002111CFCF0AC08091A302882361F085301A
:1045A00061F08091E80083FD0AC08091E80082FFFD
:1045B000F2CF80E0089582E0089583E0089581E0DD
:1045C00008952091AA023091AB022617370748F0D0
:1045D0006115710539F42091E8002E772093E800E9
:1045E00001C0B901FC0120E06115710591F18091D4
:1045F000A302882309F440C0853009F43FC08091AC
:10460000E80083FD3DC08091E80082FD2FC08091CD
:10461000E80080FFE9CF2091F3008091F20090E064
:10462000922B6115710559F08830910540F4249161
:104630002093F1003196615071090196F2CF21E08B
:10464000089709F020E08091E8008E778093E800D9
:10465000CBCF2111CCCF0AC08091A302882361F077
:10466000853061F08091E80083FD0AC08091E80008
:1046700082FFF2CF80E0089582E0089583E00895FC
:1046800081E00895982F973068F59093E900981786
:1046900039F07091EC002091ED005091F00003C0D2
:1046A000242F762F50E021FD02C09F5FECCF309188
:1046B000EB003E7F3093EB003091ED003D7F309377
:1046C000ED003091EB0031603093EB007093EC0023
:1046D0002093ED005093F0002091EE0027FDE5CFF0
:1046E00080E008958F708093E90081E008958091C3
:1046F000A40287FF11C08091E80082FD05C080916F
:10470000A3028111F8CF11C08091E8008B770BC014
:104710008091A302882349F08091E80080FFF8CFC0
:104720008091E8008E778093E80008952091E4005E
:104730003091E50095E64091EC00842F817040FFB8
:1047400023C08091E80080FD1DC08091A3028823D2
:1047500099F0853099F08091EB0085FD11C0409172
:10476000E4005091E5002417350729F3915011F02A
:104770009A01E1CF84E0089582E0089583E00895EE
:1047800081E0089580E008954091E80042FFDDCF88
:1047900008950E9437240E943F24E0EEF0E08081DB
:1047A00081608083E8EDF0E080818F77808319BCA1
:1047B000A7EDB0E08C918E7F8C9380818F7E80837B
:1047C0001092A20208950F931F93CF93DF930E943C
:1047D00037240E943F24C8EDD0E088818F778883FA
:1047E00088818068888388818F7D888319BC109236
:1047F000A30210929F021092A1021092A00200EE5A
:1048000010E0F80180818B7F8083888181608883BC
:1048100042E060E080E00E944223E1EEF0E080812F
:104820008E7F8083E2EEF0E08081816080838081F2
:1048300088608083F80180818E7F80838881806199
:104840008883DF91CF911F910F910895E8EDF0E0FB
:1048500080818F7E8083E7EDF0E0808181608083BE
:1048600084E082BF81E08093A2020C94E323E8ED10
:10487000F0E080818E7F80831092E2000895109294
:10488000DA001092E10008951F920F920FB60F9276
:1048900011242F933F934F935F936F937F938F9345
:1048A0009F93AF93BF93EF93FF938091E10082FFBB
:1048B0000BC08091E20082FF07C08091E1008B7FF6
:1048C0008093E1000E94BA268091DA0080FF1FC029
:1048D0008091D80080FF1BC08091DA008E7F80938A
:1048E000DA008091D90080FF0DC080E189BD82E1AE
:1048F00089BD09B400FEFDCF81E08093A3020E9430
:104900008C2005C019BC1092A3020E949A208091AD
:10491000E10080FF19C08091E20080FF15C0809106
:10492000E2008E7F8093E2008091E20080618093BC
:10493000E2008091D80080628093D80019BC85E0A5
:104940008093A3020E949F208091E10084FF30C0E9
:104950008091E20084FF2CC080E189BD82E189BDA5
:1049600009B400FEFDCF8091D8008F7D8093D800E0
:104970008091E1008F7E8093E1008091E2008F7E44
:104980008093E2008091E20081608093E200809158
:104990009F02882311F084E007C08091E30087FD27
:1049A00002C081E001C083E08093A3020E94A7209F
:1049B0008091E10083FF29C08091E20083FF25C040
:1049C0008091E100877F8093E10082E08093A302E1
:1049D00010929F028091E1008E7F8093E100809190
:1049E000E2008E7F8093E2008091E20080618093FC
:1049F000E20042E060E080E00E9442238091F0000B
:104A000088608093F0000E949D20FF91EF91BF91FC
:104A1000AF919F918F917F916F915F914F913F9156
:104A20002F910F900FBE0F901F9018951F920F920D
:104A30000FB60F9211242F933F934F935F936F9371
:104A40007F938F939F93AF93BF93CF93DF93EF9316
:104A5000FF93C091E900CF708091EC00D82FD17006
:104A600080FDD0E81092E9008091F000877F80936C
:104A7000F00078940E945A251092E9008091F0008D
:104A800088608093F000CD2BCF70C093E900FF9138
:104A9000EF91DF91CF91BF91AF919F918F917F91D6
:104AA0006F915F914F913F912F910F900FBE0F909B
:104AB0001F9018951F93CF93DF93CDB7DEB7AA97BA
:104AC0000FB6F894DEBF0FBECDBFE4EAF2E08091EE
:104AD000F100819322E0EC3AF207C9F70E94C52069
:104AE0008091E80083FF2EC18091A4029091A502DD
:104AF000492F50E04A30510508F024C1FA01EE591F
:104B0000FF4F0C942E27803821F0823809F01AC10B
:104B100008C08091A0029091A102992389F082603F
:104B20000FC08091A8028F70873008F00BC180936E
:104B3000E9008091EB0085FB882780F91092E9005D
:104B40009091E800977F9093E8008093F100109295
:104B5000F100D1C0282F2D7F09F0F4C0882319F06F
:104B6000823061F0EFC08091A602813009F0EAC086
:104B7000933009F080E08093A1022EC08091A602BC
:104B800081112AC08091A8028F702FEF280F263044
:104B900008F0D8C08093E9002091EB0020FF1CC0F2
:104BA000933021F48091EB00806214C09091EB006F
:104BB00090619093EB0021E030E0A90102C0440F26
:104BC000551F8A95E2F74093EA001092EA0080911F
:104BD000EB0088608093EB001092E9008091E80080
:104BE000877F8093E8000E947723ACC08111AAC020
:104BF0001091A6021F778091E3008078812B80932B
:104C0000E3008091E800877F8093E8000E9477238B
:104C10008091E80080FFFCCF8091E3008068809362
:104C2000E300111102C082E001C083E08093A3027F
:104C300089C08058823008F085C08091A60290918A
:104C4000A7028C3D53E0950779F583E08A838AE2D9
:104C500089834FB7F894DE01139620E03EE051E2DD
:104C6000E32FF0E050935700E49120FF03C0E2955A
:104C7000EF703F5FEF708E2F90E0EA3010F0C79634
:104C800001C0C0968D939D932F5F243149F74FBF8C
:104C90008091E800877F8093E8006AE270E0CE01AF
:104CA00001960E94832216C06091A8027091A90209
:104CB000AE014F5F5F4F0E94C721BC01892B09F4F1
:104CC00041C09091E800977F9093E80089819A8194
:104CD0000E94E1228091E8008B778093E80032C047
:104CE000803881F58091E800877F8093E80080918B
:104CF0009F028093F1008091E8008E7772CF81113E
:104D000021C08091A6029091A70299270297D4F41E
:104D10008091E800877F8093E8008091A6028093CD
:104D20009F020E94772380919F02811106C080918B
:104D3000E30087FD02C081E001C084E08093A3020C
:104D40000E94B1208091E80083FF0AC08091E800B2
:104D5000877F8093E8008091EB0080628093EB0076
:104D6000AA960FB6F894DEBF0FBECDBFDF91CF91EC
:104D70001F9108950895CF938091A3028823A1F0F5
:104D8000C091E900CF709091EC00892F817090FD67
:104D900080E8C82B1092E9008091E80083FD0E9412
:104DA0005A25CF70C093E900CF91089587FB082E54
:104DB000062687FD819567FD61950E9465270EF4A3
:104DC000919507FC81950895AA1BBB1B51E107C073
:104DD000AA1FBB1FA617B70710F0A61BB70B881F8B
:104DE000991F5A95A9F780959095BC01CD0108951A
:104DF00097FB072E16F4009407D077FD09D00E9488
:104E0000E42607FC05D03EF4909581959F4F0895C8
:104E1000709561957F4F0895A1E21A2EAA1BBB1BC6
:104E2000FD010DC0AA1FBB1FEE1FFF1FA217B30776
:104E3000E407F50720F0A21BB30BE40BF50B661F8C
:104E4000771F881F991F1A9469F760957095809550
:104E500090959B01AC01BD01CF010895EE0FFF1F9E
:104E60000590F491E02D09940E943C27332312F41D
:104E70008A1B9B0B0C944D27A29FB001B39FC001CE
:104E8000A39F700D811D1124911DB29F700D811D76
:104E90001124911D08950E943C27B7FF0895821B9D
:104EA000930B08950E943C27A59F900DB49F900DF1
:104EB000A49F800D911D11240895B7FF0C945227D3
:104EC0000E945227821B930B0895991B79E004C01E
:104ED000991F961708F0961B881F7A95C9F7809539
:104EE0000895FC014150504030F001900616D1F772
:104EF0003197CF010895882799270895FB01DC0198
:104F000004C08D910190801921F441505040C8F7A0
:104F1000881B990B0895F999FECF92BD81BDF89A2F
:104F2000992780B50895A6E1B0E044E050E00C94E4
:104F3000C527A8E1B0E042E050E00C94C527262F39
:104F4000F999FECF92BD81BDF89A019700B402167F
:104F500039F01FBA20BD0FB6F894FA9AF99A0FBE2D
:104F600008950396272F0E94A0270E949F27252F90
:104F70000E94A027242F0C94A0270196272F0E947F
:104F8000A0270C949F27DC01CB01FC01F999FECFEF
:104F900006C0F2BDE1BDF89A319600B40D924150C1
:0A4FA0005040B8F70895F894FFCFD1
:104FAA00C8001902280850011E0A14010101020052
:104FBA000C000C0C01191A1B1C1D1E1F2021220A91
:104FCA00202D200E20882084200D2001E200E900F7
:104FDA00EA00B500B600B700CD008301CC008A0113
:104FEA0092019401210223022402250226022702A9
:104FFA002A02B300B4006F007000818283E200E9E4
:10500A0000EA00B500B600B700CD008301CC008AE3
:10501A000192019401210223022402250226022779
:10502A00022A02B300B4006F007000818283313219
:10503A000001020202020606060909090909090F06
:10504A000F0F0F0F0F151515181919191919191905
:10505A00191919232400FF0100010000FFFF0000B5
:06506A00010001FF00003F
:00000001FF
